:100000000C9410050C942D050C942D050C942D05C5
:100010000C942D050C942D050C942D050C942D0598
:100020000C942D050C942D050C94832C0C94552DBB
:100030000C948A270C942D050C942D050C942D05F9
:100040000C942D050C942D050C942D050C942D0568
:100050000C942D050C9412280C942D050C942D0550
:100060000C942D050C942D050C942D050C942D0548
:100070000C942D050C942D050C942D050C942D0538
:100080000C942D050C942D050C942D050C942D0528
:100090000C942D050C942D050C942D050C942D0518
:1000A0000C942D050C942D050C942D057D087D08D0
:1000B000A908A90811092F09470A470A3A09D309CB
:1000C000E409E409C22DE92DE12EE92DE12E352EBA
:1000D000582EE12EAF2EBE2E2020202020202000E2
:1000E0005343524C4B00202020202020200043412D
:1000F000505320002020202020004E4C434B200055
:10010000556E64656600464E00004C657427730AA0
:100110006275696C640A736F6D652D0A7468696E27
:10012000670A746F2D0A6765742D0A68657221006D
:100130002400250026002100220023001E001F00AD
:10014000200001512700370001004A004B00010048
:100150004D004E00010001000100010001002800D7
:1001600000047F3F1F643214643214783C1E1E1456
:100170000A052223252628292A2C2D2F3032333513
:1001800036383A3B3D3E4042434547494A4C4E5043
:1001900051535557595A5C5E6062646668696B6D6D
:1001A0006F71737577797B7D7F81838587898A8C71
:1001B0008E90929496989A9C9E9FA1A3A5A7A8AA78
:1001C000ACAEAFB1B3B4B6B8B9BBBCBEBFC1C2C3AD
:1001D000C5C6C7C9CACBCCCDCED0D1D2D2D3D4D547
:1001E000D6D7D7D8D9D9DADADBDBDBDCDCDCDCDC70
:1001F000DDDDDDDDDCDCDCDCDCDBDBDBDADAD9D948
:10020000D8D7D7D6D5D4D3D2D2D1D0CECDCCCBCAD5
:10021000C9C7C6C5C3C2C1BFBEBCBBB9B8B6B4B3FB
:10022000B1AFAEACAAA8A7A5A3A19F9E9C9A989691
:100230009492908E8C8A89878583817F7D7B797764
:100240007573716F6D6B6968666462605E5C5A5944
:1002500057555351504E4C4A4947454342403E3D05
:100260003B3A3836353332302F2D2C2A2928262593
:100270002322FFAA7F554000010101010101010174
:100280000102020202020202020203030303030349
:100290000303040404040404040505050505060617
:1002A00006060607070707070808080809090909D5
:1002B0000A0A0A0B0B0B0C0C0C0D0D0D0E0E0E0F7B
:1002C0000F0F10101111111212131314141515160B
:1002D000161717181819191A1A1B1B1C1D1D1E1E7C
:1002E0001F202021222223242425262627282929CD
:1002F0002A2B2C2D2D2E2F303132323334353637F8
:1003000038393A3B3C3D3E3F4041424344454647F5
:1003100048494A4C4D4E4F50515354555658595ACE
:100320005B5D5E5F616264656668696B6C6D6F7072
:1003300072737577787A7B7D7E8082838587888AE1
:100340008C8E8F91939596989A9C9EA0A2A3A5A718
:10035000A9ABADAFB1B3B5B7BABCBEC0C2C4C6C914
:10036000CBCDCFD1D4D6D8DBDDDFE2E4E7E9EBEECD
:10037000F0F3F5F8FAFDFF00AE00AF00DA0281FFFE
:10038000D9F1DB20A4A62EAF00A0C000A1C800AE0A
:10039000D580A81FD300408D14200007087F0807D0
:1003A000003E5B4F5B3E003E6B4F6B3E001C3E7C55
:1003B0003E1C00183C7E3C18001C577D571C001C3E
:1003C0005E7F5E1C0000183C180000FFE7C3E7FFDB
:1003D00000001824180000FFE7DBE7FF0030483A70
:1003E000060E00262979292600407F0505070040D2
:1003F0007F05253F005A3CE73C5A007F3E1C1C0805
:1004000000081C1C3E7F0014227F2214005F5F0046
:100410005F5F0006097F017F00006689956A0060C2
:10042000606060600094A2FFA2940008047E04084B
:100430000010207E20100008082A1C0800081C2A32
:100440000808001E10101010000C1E0C1E0C0030AE
:10045000383E383000060E3E0E0600000000000058
:100460000000005F000000000700070000147F1478
:100470007F1400242A7F2A120023130864620036A6
:100480004956205000000807030000001C224100CC
:10049000000041221C00002A1C7F1C2A0008083E84
:1004A00008080000807030000008080808080000F4
:1004B00000606000002010080402003E5149453EE3
:1004C0000000427F400000724949494600214149ED
:1004D0004D33001814127F10002745454539003C64
:1004E0004A49493100412111090700364949493635
:1004F00000464949291E0000001400000000403455
:100500000000000008142241001414141414000008
:1005100041221408000201590906003E415D594E6E
:10052000007C1211127C007F49494936003E41414E
:100530004122007F4141413E007F49494941007FBE
:1005400009090901003E41415173007F0808087FF5
:100550000000417F4100002040413F01007F08141E
:100560002241007F40404040007F021C027F007F0C
:100570000408107F003E4141413E007F0909090601
:10058000003E4151215E007F091929460026494954
:1005900049320003017F0103003F4040403F001FFC
:1005A0002040201F003F4038403F00631408146380
:1005B000000304780403006159494D4300007F4162
:1005C000414100020408102000004141417F000425
:1005D00002010204004040404040000003070800C0
:1005E000002054547840007F284444380038444464
:1005F000442800384444287F0038545454180000DC
:10060000087E09020018A4A49C78007F08040478DE
:100610000000447D4000002040403D00007F102845
:1006200044000000417F4000007C04780478007C96
:100630000804047800384444443800FC1824241882
:100640000018242418FC007C0804040800485454B2
:1006500054240004043F4424003C4040207C001CFF
:100660002040201C003C4030403C004428102844DE
:10067000004C9090907C004464544C440000083638
:100680004100000000770000000041360800000231
:1006900001020402003C2623263C0000000000006A
:1006A00000404040F0F8F8FF38FFF8F83FF8F8FF56
:1006B00038FFF8F8F040404000000000000080C023
:1006C000C0C0800000C0C08000000080C0C000C06A
:1006D000C0000080C0C00000000000C0C0C0C0C09A
:1006E00000C0C0000000000000000000000000008A
:1006F00000000000000000000000000000000000FA
:1007000000000000000000000000000000000000E9
:1007100000000000000000000000C0F0F8FC3E1ED9
:1007200006010000007F4141417F007F4141417F40
:10073000000080C0E07E5B4F5BFEC00000C000DCBC
:10074000D7DEDEDED7DC00C00000000000000000C5
:100750000000000000000000000000000000000099
:1007600000494949FFFFFFFFE0DFBFBF00BFBFDF18
:10077000E0FFFFFFFF49494900000000001F3F6004
:1007800060E0BF1F007F7F071E381E077F7F007F4E
:100790007F0E1F3B716000000000007F7F0C0C0C7F
:1007A000007E7E007F7E0303007F7E03037E7E0348
:1007B000037F7E000F3E703C063C703E0F00327B94
:1007C00049493F7E007F7E0303001E3F69696F2613
:1007D00000000000000000000000030F1F3F3C78F5
:1007E00070600000007F4141417F007F4141417FB7
:1007F00000307B7F7830202030787F3B0003000F73
:100800007F0F0F0F7F0F00030000000000000000AB
:1008100000000000000000000000000000000000D8
:1008200000010101070F0F7F0F7F0F0F7E0F0F7F5A
:100830000F7F0F0F07010101000000000000000002
:1008400000000101000000000000000000000000A6
:100850000000000000000000000000000000000098
:100860000000000000000000000000000000000088
:100870000000000000000000000000000000000078
:100880000000000000000000000000000000000068
:100890000000000000000000000000000000000058
:1008A0000000000000000000000000000000000048
:1008B0000000000000000000000000000000000038
:1008C0000000000000000000000000000000000028
:1008D00000000000000000000000000E0352006F46
:1008E000004D00610063002B0000002603540068E7
:1008F00000650052006F00790061006C00530077C2
:100900000065006100740073006800690072007483
:100910000000000403090409023B00020100A0FAE0
:100920000904000001030101000921110100012255
:1009300040000705810308000109040100010300CC
:100940000000092111010001227B0007058203201C
:10095000000112010002000000084B4B02000100E0
:100960000102000105010902A10185020901A1009E
:10097000050919012908150025019508750181024D
:100980000501093009311581257F95027508810619
:1009900009381581257F950175088106050C0A38EF
:1009A000021581257F950175088106C0C0050109E2
:1009B00080A101850319012AB700150126B700950A
:1009C0000175108100C0050C0901A1018504190100
:1009D0002AA002150126A002950175108100C0050C
:1009E000010906A101050719E029E7150025019570
:1009F0000875018102950175088101050719002913
:100A0000FF150026FF0095067508810005081901ED
:100A10002905950575019102950175039101C000A5
:100A200011241FBECFEFDAE0DEBFCDBF11E0A0E0A2
:100A3000B1E0EEE1F0E602C005900D92AA3DB107EB
:100A4000D9F724E0AAEDB1E001C01D92A43EB2079F
:100A5000E1F70E9448160C940D300C94000083E0DE
:100A60000895CF9360E08AE091E00E946B2160914D
:100A7000E8017091E9018091EA019091EB010E94F7
:100A80003F06882331F0813041F460E086E091E058
:100A900007C060E089E091E003C060E080E091E0A1
:100AA0000E947D210E94B226C82F80FD03C084EFE2
:100AB00090E002C08AEF90E060E00E946B21C1FDEF
:100AC00003C086EE90E002C08EEE90E060E00E94EF
:100AD0006B21C2FD03C088ED90E002C080EE90E083
:100AE00060E00E946B2180E0CF91089581E008953D
:100AF00081E008950C94780508950C947C051F936B
:100B0000CF93DF9300D000D01F92CDB7DEB74983DB
:100B10005A836B833091DD0189819A81311114C030
:100B2000662359F0222349F00E94840C182F682F65
:100B300089819A810E942D0C03C00E94580C182FA5
:100B400069817A81812F04C00E94840C69817A8135
:100B50000F900F900F900F900F90DF91CF911F91FA
:100B60000C94D313FC01262F408151816281738143
:100B700084810C947F0581E00895CF93DF93EC018D
:100B800060E00E94B205BE01DF91CF910C947D051B
:100B90000C9419150C94151508950E94D70A0E94FB
:100BA000CC052FEF84E39CE0215080409040E1F79A
:100BB00000C000000C9438280F931F93CF93DF934D
:100BC0008C0161E00E94B205EC01B8010E947A0537
:100BD000882309F444C0B801CE010E944725882328
:100BE000F1F1B801CE010E94F0228823C1F1B801D1
:100BF000CE010E94A324882391F1B801CE010E9466
:100C0000091F882361F1F8018281882309F1CB351E
:100C10008DE5D807C1F050F4C115FCE5DF0781F080
:100C2000CF3DDC45A9F40E94BB1119C0CC35EDE5E0
:100C3000DE0761F0CD35DD4559F40E94FE1008C095
:100C40000E94CD050CC00E94071102C00E940A112B
:100C5000C801DF91CF911F910F910C94760580E030
:100C6000DF91CF911F910F9108950E946D270E94EF
:100C7000A0060C94A6220E94A3060C947327CF9280
:100C8000DF92EF92FF926C01EE24FF24C114D10495
:100C9000E104F10421F0C701B60120E101C020E028
:100CA000C72ED82EE92EFF24C114D104E104F1048B
:100CB00019F0285FC701B6016B017C0154E0F6947E
:100CC000E794D794C7945A95D1F7C114D104E1049D
:100CD000F10419F02C5FC701B6016B017C0142E001
:100CE000F694E794D794C7944A95D1F7C114D104E8
:100CF000E104F10419F02E5FC701B601DC01CB015C
:100D0000B695A79597958795892B8A2B8B2B09F0FC
:100D10002F5F822FFF90EF90DF90CF90089508957E
:100D20000C948F0681E008950C9492060895CF9359
:100D3000C82F0E9490068C2F0E949406CF91089590
:100D400080E00C9497060E94B2260C9497060E94AD
:100D5000B2269091DC01891721F08093DC010C947C
:100D600097060895CF93DF93CDB7DEB72B970FB6D5
:100D7000F894DEBF0FBECDBF4F83588769877A874F
:100D80008B8761110E944A109E012F5F3F4F86E0C2
:100D9000F90111928A95E9F785E0FE013796D901AC
:100DA00001900D928A95E1F789819A814C815D814C
:100DB000452B31F09F3F31F491E08F3F19F403C090
:100DC00091E001C090E090FF09C049815A816B8198
:100DD0007C818D819E810E946B0F05C0C9010E949C
:100DE000BB058111F2CF2B960FB6F894DEBF0FBE74
:100DF000CDBFDF91CF910895FC01808191810E9448
:100E0000C60C0895CF93882309F4A4C0C82F823854
:100E1000C1F40E94B22681FD9DC069E38091020168
:100E2000909103010E9445270E946C102FEF81EEE4
:100E300094E0215080409040E1F700C0000069E359
:100E400019C0833801F50E94B22680FD83C063E596
:100E500080910201909103010E9445270E946C102D
:100E60002FEF81EE94E0215080409040E1F700C0E8
:100E7000000063E580910201909103010E944727E1
:100E8000CF910C946C108438C1F40E94B22682FD7C
:100E900061C067E480910201909103010E9445279F
:100EA0000E946C102FEF81EE94E021508040904022
:100EB000E1F700C0000067E4DDCF8CEF8C0F813AD2
:100EC000D0F46C2F80910201909103010E940F27B2
:100ED000882349F06C2F80910201909103010E94B8
:100EE00047270E946C106C2F8091020190910301A2
:100EF0000E944527C5CF80E28C0F883048F4C77028
:100F000081E001C0880FCA95EAF70E942D10B8CF82
:100F1000EBE5EC0FE33040F4F0E0EF59FE4F808159
:100F200090E0CF910C94D726E8E5EC0FE73150F430
:100F3000F0E0EE0FFF1FED5CFE4F80819181CF91BD
:100F40000C94ED26CD3E30F08C2F0E94CD16CF9123
:100F50000C949F17CF910895882309F464C08238B8
:100F600079F40E94B22681FF5EC069E3809102019C
:100F7000909103010E9445270E946C1069E310C004
:100F80008338B1F40E94B22680FF4DC063E58091A2
:100F90000201909103010E9445270E946C1063E5B5
:100FA00080910201909103010E9447270C946C10DC
:100FB000843879F40E94B22682FF35C067E48091BC
:100FC0000201909103010E9445270E946C1067E482
:100FD000E7CF9CEF980F913A10F4682FE1CF90E2A1
:100FE000980F983050F4877091E001C0990F8A955E
:100FF000EAF7892F0E943310D9CF9BE5980F9330E1
:1010000020F480E090E00C94D72698E5980F973173
:1010100020F480E090E00C94ED268D3E20F00E94BC
:1010200028170C949F1708951F93CF93DF93182FC1
:10103000EB010E940207209741F08FE99FE00197A2
:10104000F1F700C000002197F6CF812FDF91CF91FB
:101050001F910C94AC07893319F060E070E002C076
:1010600060E570E00C941408882321F00E942D1094
:101070000C946C100895882321F00E9433100C9476
:101080006C100895CF92DF92EF92FF920F931F930F
:10109000CF93DF937C01D62FC72FFC0112810581EE
:1010A00002950F700E9423108823B9F01123A9F034
:1010B0008C2F807F803421F080E28D0F883068F0A3
:1010C0008091B30282FD09C082E00E94CC100E9490
:1010D000231091E0D82ED92601C0D12CCC2EC29459
:1010E0008FE0C8228C2D90E08C30910508F0CFC1A4
:1010F000FC01EA5AFF4F0C946B2F8C2F807FCF702E
:10110000882311F0C295C07F112399F0CC2309F4F4
:10111000AAC180E28D0F883010F0D11104C08C2F4D
:101120000E942D1003C08C2F0E943D100E946C1055
:101130009AC18D2F0E94AC07CC2309F4A8C180E28C
:101140008D0F883038F1DD2329F18C2F0E94431058
:1011500024C08C2F807FCF70803211F0C295C07F69
:10116000DD2319F0D130A1F13DC08091B30282FF9F
:1011700017C0112349F0CC2329F08C2F0E942D1089
:101180000E946C1080E070C180E00E94AC07CC230C
:1011900009F47DC18C2F0E9433100E946C1077C11E
:1011A000112371F0002341F0013031F40E944D1001
:1011B0008C2B0E9455106BC10E944D108C2B1DC0B2
:1011C000002319F0013009F462C10E94621025C0A9
:1011D000112321F0063008F05AC10EC0053008F086
:1011E00056C11BC0112361F0002331F0F701858146
:1011F00080FF39C18F7085838C2F0E94340847C1CE
:10120000002359F0D93309F03FC1FFEF07EE13E097
:10121000F15000401040E1F735C18C2F0E943B088F
:1012200036C18C2F86958695837019F0813061F0D8
:101230002EC1112321F08D2F9C2F937002C080E0CE
:1012400090E00E94D7262BC1112321F08D2F9C2FD7
:10125000937002C080E090E00E94ED2620C18D2FA7
:10126000112319F00E94CD1602C00E9428170E9477
:101270009F1715C18C2F837009F047C011110BC146
:101280002D2F229526952770220F220F6D2F6F701C
:10129000862F90E0A0E0B0E0022E04C0880F991FD6
:1012A000AA1FBB1F0A94D2F7D4FF10C04FE050E032
:1012B00060E070E004C0440F551F661F771F2A9539
:1012C000D2F7409550956095709503C040E050E08E
:1012D000BA01C695C695C3708A019B01082B192BCC
:1012E0002A2B3B2BC901B801C23049F058F4C13058
:1012F00019F00E94430BCFC00E94310BCCC00E945A
:10130000550BC9C00E942F0BC6C0112319F08C2F9A
:10131000817001C08695882309F4BDC02D2F2295C8
:1013200026952770220F220F6D2F6F70862F90E069
:10133000A0E0B0E0022E04C0880F991FAA1FBB1FB7
:101340000A94D2F7D4FF10C04FE050E060E070E0A4
:1013500004C0440F551F661F771F2A95D2F740958A
:1013600050956095709503C040E050E0BA01C69575
:10137000C695C3708A019B01082B192B2A2B3B2B86
:10138000C901B801C23049F058F4C13019F00E94C7
:10139000080C81C00E94F60B7EC00E941A0C7BC014
:1013A0000E94690B78C0CF70112339F08C2F0E94F6
:1013B0008F0B8D2F0E9434086EC08D2F0E943B082A
:1013C0008C2F0E94B00B67C0D23F21F128F4D03F90
:1013D00041F0D13FC1F043C0D33F19F1D43F79F080
:1013E0003EC0112341F0053008F051C08C2F8F71A1
:1013F0000E94D50B4CC0063008F049C0F7CF809151
:10140000B30282FF18C0112339F08C2F8F710E9414
:101410008F0B3DC01123C9F38C2F8F710E94B00B2D
:1014200036C0112329F08C2F8F710E947A0B2FC0A8
:101430000E94750B2CC0112349F0CF718C2F0E9494
:101440008F0B63E08C2F0E94B11021C081E00E94BD
:10145000CC100230E0F082E00E94CC1018C01123C2
:1014600031F0002391F28D2F0E94020710C000235B
:1014700099F2D93349F41FEF27EE33E011502040A1
:101480003040E1F700C000008D2F0E94AC0788EFCC
:101490008C0D843020F40E94B2260E949706DD2035
:1014A000C9F00E941F1080FD15C0F70112820E9432
:1014B00019100E948F0BC7010E948B0A0E941910FD
:1014C000DF91CF911F910F91FF90EF90DF90CF9020
:1014D0000C94B00BDF91CF911F910F91FF90EF9083
:1014E000DF90CF9008950F931F93CF93DF93EC017C
:1014F000688179818A810E94D10C8C010E942C0C18
:101500000E941D0BB801CE010E944208DF91CF91CD
:101510001F910F910895CF93DF93EC0198818981FA
:101520002B813C81232B31F08F3F31F481E09F3FB1
:1015300019F403C081E001C080E080FD1DC0CE0130
:101540000E94DC05811110C00E9423108823A1F0A5
:101550008A81882389F08091B30282FD0DC082E0E8
:10156000DF91CF910C94CC10CE010E94730ACE0172
:10157000DF91CF910C94BD05DF91CF91089580E06C
:1015800090E00E94D72680E090E00E94ED260E9425
:101590004A100E946C100E94D0180C949F178091E2
:1015A0000201909103010E9449270C94BF0A0E94F6
:1015B0003A100C94CF0A92959F70963079F010F4FF
:1015C000925001C09A50923068F4803F69F018F44C
:1015D000883E40F409C0843F29F406C0883E20F0CC
:1015E000813F11F080E0089581E00895FC01808141
:1015F00091810E94C60C0E94DB0A0895CF93DF936D
:1016000000D000D01F92CDB7DEB70F900F900F9093
:101610000F900F90DF91CF910895CF93DF9300D07B
:1016200000D000D0CDB7DEB726960FB6F894DEBF57
:101630000FBECDBFDF91CF910895089508950C940A
:101640001E0B0C941F0B0E94210B6093EC017093F6
:10165000ED018093EE019093EF010C94BF0A0C947E
:10166000230B0F931F930091EC011091ED0120913A
:10167000EE013091EF01602B712B822B932B1F9188
:101680000F910C94230B0F931F930091EC01109179
:10169000ED012091EE013091EF016023712382234F
:1016A00093231F910F910C94230B0F931F93009181
:1016B000EC011091ED012091EE013091EF016027D6
:1016C0007127822793271F910F910C94230B0C9461
:1016D0001E0B0E94670B6093E8017093E9018093F1
:1016E000EA019093EB010C94BF0A60E070E0CB013B
:1016F0000C94690B0F931F9341E050E060E070E0A1
:101700008A019B0104C0000F111F221F331F8A95FD
:10171000D2F7C901B8011F910F910C94690B0F9377
:101720001F9341E050E060E070E004C0440F551F9B
:10173000661F771F8A95D2F78091E8019091E901A1
:10174000A091EA01B091EB018A019B01082B192BB2
:101750002A2B3B2BC901B8011F910F910C94690BE7
:101760000F931F9341E050E060E070E004C0440F2D
:10177000551F661F771F8A95D2F740955095609543
:1017800070958091E8019091E901A091EA01B091F2
:10179000EB018A019B01082319232A233B23C9015A
:1017A000B8011F910F910C94690B0F931F9341E0A7
:1017B00050E060E070E004C0440F551F661F771FC3
:1017C0008A95D2F78091E8019091E901A091EA0110
:1017D000B091EB018A019B01082719272A273B2793
:1017E000C901B8011F910F910C94690B0F931F93BE
:1017F0000091E8011091E9012091EA013091EB019B
:10180000602B712B822B932B1F910F910C94690BE2
:101810000F931F930091E8011091E9012091EA01D3
:101820003091EB0160237123822393231F910F9149
:101830000C94690B0F931F930091E8011091E9013B
:101840002091EA013091EB016027712782279327CD
:101850001F910F910C94690B0895292F220F920F5D
:10186000890FE82FE695E695E695877051E001C06F
:10187000550F8A95EAF785E0E89FF0011124E252BE
:10188000FE4F20E030E070E04081CB01022E02C02C
:10189000969587950A94E2F7817081958427852330
:1018A000842781932F5F3F4F2530310569F70895D5
:1018B000292F220F920F890F682F669566956695DE
:1018C000982F977085E0689FB001112440E050E0A8
:1018D00080E0FB01E40FF51FE252FE4F208130E073
:1018E000092E02C0369527950A94E2F72170332716
:1018F000042E01C0220F0A94EAF7822B4F5F5F4F3C
:101900004530510531F70895BF92CF92DF92EF92A3
:10191000FF920F931F93CF93DF938C01C090E80148
:10192000D090E901E090EA01F090EB018091EC01A8
:101930009091ED01A091EE01B091EF01C82AD92A52
:10194000EA2AFB2ACFE1D0E0D701C6010C2E04C061
:10195000B695A795979587950A94D2F780FD04C010
:10196000219790F7B12C07C0BC2EB8018C2F0E9494
:10197000E9130197A9F38B2DDF91CF911F910F915F
:10198000FF90EF90DF90CF90BF900895CF93DF93BB
:10199000EC010E94840CBE010E94E913DF91CF91FB
:1019A00008951F93CF93DF93EB019091DD0199236D
:1019B00021F0CB010E94C60C13C0882349F0CB0153
:1019C0000E94840C182F682FCE010E942D0C04C099
:1019D000CB010E94580C182FBE01812F0E94E913E1
:1019E000DF91CF911F9108951F93CF93DF93C09103
:1019F000F00116E08091F101C81799F0D0E01C9F2A
:101A0000F0011D9FF00D1124EE50FE4F40815181D9
:101A100062817381848195810E940D0B2196C7702C
:101A2000E9CFDF91CF911F9108954091220250910B
:101A300023026091240270912502809126029091E8
:101A400027020C940D0BEF92FF920F931F93CF93ED
:101A5000DF938091270282958F7009F065C0809195
:101A60002402882309F460C08091F001F090F10114
:101A700010912202009123026091250270912602AA
:101A800091E01F3F09F090E0C0910001D091010169
:101A9000292F96E0E92E8F1509F446C061157105CE
:101AA00021F00F3F21F030E003C031E001C0322FC0
:101AB00090E030FD36C0E89EF001E99EF00D112463
:101AC000DF01AE50BE4F11963C911197301329C0E3
:101AD0003C91311326C012963C911297311121C0CE
:101AE00013964D915C911497461B570B4C175D074D
:101AF000C0F4809127028F70806180932702E950A3
:101B0000FE4F80818F708061808382E292E00E942C
:101B10008B0ADF91CF911F910F91FF90EF900C9462
:101B2000F40C01968770B7CFDF91CF911F910F9181
:101B3000FF90EF9008959F92AF92BF92CF92DF9265
:101B4000EF92FF920F931F93CF93DF93CDB7DEB742
:101B500061970FB6F894DEBF0FBECDBF8C0185E054
:101B6000F801DE011D9601900D928A95E1F7D801EA
:101B70001296EC9090912202E0912302209125028E
:101B8000309126022115310531F0EF3F31F481E02B
:101B90009F3F19F403C081E001C080E0B82FB1700D
:101BA0009B2E80FD47C1D8014C9111965C911197F5
:101BB0001396AD90BC90149782E2C82E82E0D82E86
:101BC000F0902402B501621B730B2091000130914B
:101BD0000101FF2009F4D9C0809127026217730721
:101BE00008F095C0282F207F09F052C05E1313C063
:101BF000491311C0FE2CE1100EC08F7080618093DC
:101C000027020E94150DC6010E948B0A80912702AF
:101C1000F80185834DC1AB2831F05F3F31F481E09D
:101C20004F3F19F403C081E001C080E080FD03C094
:101C300081E08E2502C080E090E0F82FF170FF2E49
:101C400080FF1CC08091F0012091F10136E08217E5
:101C500009F40BC190E0389FF001399FF00D112479
:101C6000EE50FE4F6181561306C06081461303C0DB
:101C70006281E61203C001968770E9CFFE2CEE2048
:101C800009F416C18091270281608093270254C015
:101C90005E1306C0491304C0E11002C0F80199C0E8
:101CA000C8010E94F60A882361F1EE2051F12091CB
:101CB0002702822F82958F7090E0029774F08091B6
:101CC00022029091230298878F831986BB86AA8669
:101CD0002C87CE0107960E948B0A86E0F801A2E2CB
:101CE000B2E001900D928A95E1F70E94230D0E94C7
:101CF000150D0AC05E1711F1C8010E94F60A811184
:101D00002CC0C8010E948B0AFF24F394D1C0282F55
:101D1000207F81F77A2DB98AA88A6E2D89890E9441
:101D2000FE0A82E292E00E948B0A86E0D6011D92B2
:101D30008A95E9F70E94150DF12CBAC04913DCCF42
:101D4000E110DACFF8018583C8010E948B0A86E092
:101D5000D6011D928A95E9F7ABC0EE2091F2209151
:101D60002702822F82958F7090E002970CF4B5CFF6
:101D700080912202909123029A8389831B82BD82E3
:101D8000AC822E83CE010196A6CF6217730708F0AE
:101D900044C0FE2CEE2009F4B4CF5E1330C04913CA
:101DA0002EC02091270220FD21C0822F82958F70A6
:101DB000482F50E041155105C9F0F80125834F30F7
:101DC000510541F08F5F982F9295907F822F8F70F1
:101DD000892B8583C8010E948B0A86E0F801A2E264
:101DE000B2E001900D928A95E1F73CC086E0F801DF
:101DF000A2E2B2E001900D928A95E1F759C0C801C4
:101E00000E94F60A811169CF809127028160809338
:101E10002702C8010E948B0A4BC07A2DB98AA88A72
:101E20006E2D89890E94FE0A86E0D6011D928A9550
:101E3000E9F718C0EE2009F464CFC8010E94F60A41
:101E4000F82E882309F45DCF86E0F801A2E2B2E023
:101E500001900D928A95E1F782E292E00E94FC06E1
:101E60000E94230D0E94150D23C04D875E878D852E
:101E70009E850E94C60C292F22952F70223028F4AF
:101E80009F7039F0811105C00BC0243028F49F7079
:101E900049F4805E883020F0C8010E948B0A9F2C94
:101EA000F92C06C0D80115969C91907F91F7F8CF38
:101EB0008F2D61960FB6F894DEBF0FBECDBFDF91B8
:101EC000CF911F910F91FF90EF90DF90CF90BF9037
:101ED000AF909F9008951F93CF93DF93CDB7DEB758
:101EE0002C970FB6F894DEBF0FBECDBF4F83588737
:101EF00069877A878B879C87CE0107960E949B0D06
:101F00008823D1F09F8188852A853B85232B31F05A
:101F10008F3F31F481E09F3F19F403C081E001C09D
:101F200080E080FD47C04F81588569857A858B8523
:101F30009C850E940D0B3EC086E0FE013796DE01B7
:101F4000119601900D928A95E1F7FF81E8856A85E7
:101F50007B856115710531F0EF3F31F481E0FF3F82
:101F600019F403C081E001C080E080FD23C020910E
:101F7000F10130E0C9010196877099274091F00185
:101F800050E084179507F1F1F983EA837D836C8330
:101F900096E0929FD001939FB00D1124AE50BE4F9A
:101FA000FE01319601900D929A95E1F78093F1012F
:101FB0000E94F40C16E08091F0019091F1018917D4
:101FC00071F1189FC00111248E509E4F0E949B0DED
:101FD000882329F1E091F0011E9FF0011124EE50B9
:101FE000FE4F4081518162817381848195810E947D
:101FF0000D0B8091F00190E00196877099278093F6
:10200000F001D9CF0E94D70A1092F1011092F0018D
:10201000E2E2F2E086E0DF011D928A95E9F72C9674
:102020000FB6F894DEBF0FBECDBFDF91CF911F91E9
:1020300008958091300285958595859508958091C4
:1020400030028770089590913002977081E009F412
:1020500080E0089580913B02089590913B02892B86
:1020600080933B020895809590913B028923809351
:102070003B02089510923B02089590913A02892BF9
:1020800080933A020895809590913A028923809333
:102090003A02089510923A0208958091310208950B
:1020A00008950C9450100C9451109091B30292FD2D
:1020B00008C090913102981721F0809331020C945E
:1020C0005310089580913102882329F01092310233
:1020D00080E00C9453100895CF93DF93E0910201B8
:1020E000F091030180913B028083E0910201F09125
:1020F0000301908180913A02892B80838091310283
:10210000882381F0E0910201F09103019081892BF5
:10211000808380910201909103010E940327811125
:102120000E946210C0910201D091030148E050E08A
:1021300068E272E0CE010E94B82F892B69F088E036
:10214000FE01A8E2B2E001900D928A95E1F7CE017E
:10215000DF91CF910C94BE26DF91CF9108950C941E
:1021600050109091B30292FD10C098E0899F9001A9
:102170001124262B209330020E948F0B8091300275
:102180008595859585950C94AF100C948F0B1092C6
:10219000300280E00C94AF102091300280958223B1
:1021A00080933002982F977099F430E0482F082ED2
:1021B000000C550B2417350759F09091B30292FD8E
:1021C00007C08595859585950E94B00B0C94C71026
:1021D00008959091B30292FB222720F9281769F005
:1021E00080FB92F99093B3028091B2029091B30276
:1021F0000E94371182E00C94CC1008958091B302B4
:1022000082FB882780F991E089270C94E91081E00E
:102210000C94E91080E00C94E9106FEF7FEF80E000
:1022200090E00C94F72F80E090E00E94D32F21E003
:10223000893E9E4F09F020E0822F089582E090E0D1
:102240000C94C52F83E090E00C94C52FCF9384E0CD
:1022500090E00E94C52FC82F82E290E00E94C52F17
:102260002C2F30E0A901582BCA01CF910895CF93AC
:10227000C92F682F84E090E00E94D92F6C2F82E252
:1022800090E0CF910C94D92FAB01BC018FE090E08E
:102290000C94EB2FAB01BC0183E190E00C94EB2F8D
:1022A00060E070E0CB010C944A1160E070E0CB017B
:1022B0000E9444110C94501169EE7EEF80E090E092
:1022C0000E94F72F60E082E090E00E94D92F60E04A
:1022D00083E090E00E94D92F1092EC011092ED0162
:1022E0001092EE011092EF0160E084E090E00E9415
:1022F000D92F60E082E290E00E94D92F60E085E073
:1023000090E00E94D92F60E086E090E00E94D92FF3
:102310006FEF87E090E00E94D92F40E050E0BA01D3
:1023200088E090E00E94EB2F60E08DE090E00E945A
:10233000D92F40E050E0BA0188E190E00E94EB2FF5
:1023400060E087E190E00E94D92F40E050E0BA01C0
:102350008CE190E00E94EB2F60E070E080E290E082
:102360000E94F72F40E050E0BA0188E190E00E941F
:10237000EB2F0C9455110C945C11682F8EE090E0BB
:102380000C94D92F0E94F72760934802709349025A
:1023900080934A0290934B026093440270934502EB
:1023A000809346029093470208950E94F727609316
:1023B00048027093490280934A0290934B026093C3
:1023C0004002709341028093420290934302089529
:1023D00085B7806885BF85B7806885BF089581E02F
:1023E00008950C94EF1108950C94F3110C94F311CB
:1023F0000C94F6110C94F3110C94FA110C94F31143
:102400000E94E81185EC94E10E94A8260E94FE112A
:102410000C94FC110E94F4110C94F3110E94DF142F
:102420000C9496060E94E2270E94AE150E940E129E
:1024300080E00E9444200E94281E0E9443240C94A5
:10244000F8118F929F92AF92BF92CF92DF92EF924C
:10245000FF920F931F93CF93DF93CDB7DEB72A97E9
:102460000FB6F894DEBF0FBECDBF0E94C315982EE5
:1024700081110E94C2118CE3A82E82E0B82E00E0E8
:1024800010E0802E802F0E940315D82EF501C190F8
:102490005F01C826B1F40F5F1F4F0430110589F7A3
:1024A0008FEF89838A831B820E94EB278160782FBC
:1024B0009D838C8349815A816B818D810E94B206F4
:1024C0002FC080914C0281FD0E940915E12CFF2450
:1024D000F3948C2D8F21F1F00E94F111882399F053
:1024E000EE828F82DF2081E009F480E088870E94FD
:1024F000EB278160782F9A8789874E815F81688575
:102500008A850E94B206F801E45CFD4F8081F826BE
:10251000F08206C0E394FF0CF3E0EF12DACFBBCFFA
:1025200081E0911001C080E02A960FB6F894DEBFDA
:102530000FBECDBFDF91CF911F910F91FF90EF9014
:10254000DF90CF90BF90AF909F908F900895CF93E2
:10255000DF930E942112D82F0E945B1E0E945624F6
:10256000C82F81110E94D5110E94C222D11101C031
:10257000C1110E9482210E94BD17DF91CF910C945E
:10258000A706CF93DF930E94EE13EC01811521E59E
:10259000920708F045C0811530E5930708F094C014
:1025A000883E910528F5803E910508F0F8C0883AEC
:1025B000910570F4853A910508F07CC08130910551
:1025C00009F475C008F4E8C0049708F0E8C0E4C056
:1025D0008F3B910508F0E0C0C85AD0E0CC0FDD1F5A
:1025E000CC59DE4F0990D881C02DCE019464D8C05B
:1025F000811540E2940758F4811551E0950708F0E1
:10260000CEC08D3E910508F4C7C09065C9C0C11504
:1026100080E4D80708F4C0C0DF70CE01906AC0C063
:10262000811525E59207A8F4811534E5930708F094
:1026300095C0811543E5940708F07BC0811552E5EC
:10264000950708F061C0D82FCC27CE01816F906A22
:10265000A7C0C11589E5D807A0F4C11528E5D207A0
:1026600008F082C0C11536E5D30708F095C08C2F5D
:102670000E9482148F7190E0D82FCC27CE019062F7
:102680008FC0C1154AE5D40708F474C0CE01905636
:102690008115904208F080C08D2F8F710E948214A6
:1026A000DD27D0628F71AE01582BCA0179C081E05D
:1026B00090E076C0C55AD0E0CE56DE4F8881C82F54
:1026C000D0E0CE0190646CC074E0969587957A95C1
:1026D000E1F7282F23703C2F337081E090E002C097
:1026E000880F991F3A95E2F79C68AC01522B9A012A
:1026F0009C2F9F709695969550E2959FE00111242E
:10270000C9018C2B9D2B4CC08370992721E030E0B0
:1027100002C0220F331F8A95E2F79C2F969596955B
:1027200080E2989FE0011124C22BD32BCE019C683C
:1027300037C08370992721E030E002C0220F331F99
:102740008A95E2F79C2F9695969540E2949FE0013A
:102750001124C22BD32BCE019A6822C0D82FCC27AC
:10276000CE01846F906A1CC0DC2FCC27CE01806F15
:10277000906A16C08C2F8F700E94821494E0D695B8
:10278000C7959A95E1F7CF70D0E0DC2FCC27D069C0
:102790009E01282BC90104C080E090E001C0CE0159
:1027A000DF91CF910895272F30E0F901EE0FFF1F41
:1027B0002E0F3F1FF9019CE0899FE00DF11D1124B0
:1027C000E60FF11DEE0FFF1FE05DFE4F8591949126
:1027D00008950E94D3130E94C11208958238910572
:1027E00069F1B0F48133910509F46DC048F4893280
:1027F000910509F463C08A32910509F469C008950E
:102800008533910509F455C089339105B9F00895D0
:10281000833E910569F138F4803E9105B1F0823E26
:10282000910509F10895863E9105A9F1873E91052C
:10283000B9F1843E910509F064C023C02091B20231
:1028400020FD4FC021FD4DC008958091B20280FD52
:1028500044C08091B30280FF44C08091B20284FDE5
:1028600042C083EE4DC08091B20282FF38C0F5CFE6
:102870008091B20282FD33C08091B30280FD31C0ED
:10288000ECCF8091B30281FF32C08091B20284FD0F
:102890002AC087EE35C08091B20283FF26C0F5CFF3
:1028A0008091B20283FD21C08091B30281FD1FC0DF
:1028B000ECCF8091B20285FD1CC01DC08091B20298
:1028C00085FD19C016C08091B20286FD16C017C0E2
:1028D0008091B20286FD13C010C089E311C082EE60
:1028E0000FC080EE0DC080E00BC086EE09C084EE04
:1028F00007C089E205C085E303C08AE201C081E325
:1029000090E008959091B20292FF0DC0282F287197
:10291000283019F4877F846006C0282F2471243062
:1029200011F48B7F886093FF0DC0282F2871283108
:1029300019F4877E846106C0282F2471243111F494
:102940008B7E88612091B30220FF0DC0382F387133
:10295000383019F4877F816006C0382F31713130EB
:1029600011F48E7F886021FF0DC0282F2871283137
:1029700019F4877E816106C0282F2171213111F45D
:102980008E7E886194FD877E089580E008950C9482
:102990000D110E94C3158FE39CE90197F1F700C068
:1029A00000000E94C31580E00E94031580FF04C050
:1029B0000E94C7140C94382808950C94C9140E94DE
:1029C0001311811102C00E94BB110E941E1180933D
:1029D0004C020E9426119093B3028093B2020E948F
:1029E000DD140E942211682F70E080E090E00E94C8
:1029F0002F0B6091E8017091E9018091EA019091BB
:102A0000EB010C94670BE82FF0E0E854FD4F808158
:102A10000895089580EA8A95F1F7089500C0089511
:102A20000C940A1508950C9412150C9413150C941B
:102A300012150C941715F894E82FE295EF70F0E05A
:102A400031A1282F2F7081E090E001C0880F2A95D6
:102A5000EAF7982F9095932391A392A1892B82A3B3
:102A600078940895CF93DF93C8E9D1E089918F3F9F
:102A700011F00E941B1581E0CC39D807B9F786EF19
:102A80000E941B1585EF0E941B1584EFDF91CF91EB
:102A90000C941B15CF92DF92EF92FF920F931F932E
:102AA000CF93DF938C01C62FD0E0CE0188569E4F86
:102AB0007C01FC0190819F3F09F447C0D62EF89419
:102AC000E92FE295EF70F0E081A19F7021E030E006
:102AD00001C0220F9A95EAF7822B81A382A120954B
:102AE000282322A378940E940E15E5E9F1E048E935
:102AF00051E031E0C12C21912F3F89F0A22FA29506
:102B0000AF70B0E090968C9190E02F7002C09595D8
:102B100087952A95E2F780FD02C0832F01C080E0EF
:102B2000C82A330F4E175F0731F7F70180818F3FB7
:102B300011F00E941B1561E0C11001C060E08D2DF5
:102B40000E941015C00FD11FC882DF91CF911F9135
:102B50000F91FF90EF90DF90CF9008950E94321573
:102B600084E0E8EBF2E0DF01982F1D929A95E9F7F7
:102B7000E4EBF2E0DF011D928A95E9F784E00E9420
:102B800005160C94C8051F93CF93DF9300D000D097
:102B9000CDB7DEB719821A821B821C8210E0612F2A
:102BA000CE0101960E944A151F5F1430C1F744E020
:102BB00050E0BE016F5F7F4F84EB92E00E94B82F20
:102BC00011E0009709F410E0892B61F089819A8166
:102BD000AB81BC818093B4029093B502A093B602FE
:102BE000B093B702212F44E068EB72E084EB92E0EF
:102BF0000E9406160E94CA05812F0F900F900F9019
:102C00000F90DF91CF911F9108950895FF920F9338
:102C10001F93CF93DF938C01F62ED72FC42F22233F
:102C200049F081E080934F020E94EB2790934E027F
:102C300080934D0280914F028823C1F080914D0214
:102C400090914E020E940328059780F0EF2DFD2FF2
:102C5000D8014C2F50E0CD01801B910B84179507B4
:102C60001CF48D918193F7CF10924F02DF91CF9199
:102C70001F910F91FF9008950E94DB290E9412126C
:102C80000C94E7290E94EB290E94A7120C94052AB4
:102C90000E9489270E94C2290E9400120E943C16AD
:102CA0000E9442160E940A12FBCF8091560280FFBA
:102CB00006C06091090170E0660F771F26C081FF92
:102CC00004C06091090184E005C082FF07C06091E3
:102CD000090188E0689FB001112417C09091550246
:102CE0009923D1F060910801961788F72091090186
:102CF00088E0289F90011124929FA001939F500D7E
:102D0000112470E0CA010E94352F6038710540F42B
:102D10006115710519F406C068E070E0862F08950A
:102D20008FE7089581E008958091560280FF08C0E2
:102D30006091050170E0759567957595679521C05F
:102D400081FF06C06091050170E07595679519C017
:102D500082FF04C06091050170E010C090915402A0
:102D6000992399F0609104019617A0F780910501CD
:102D7000899FC001112470E00E94352F60387105D1
:102D800040F46115710519F406C061E070E0862F0A
:102D900008958FE7089581E008958D3E21F40E9403
:102DA0005516819504C08E3E29F40E9455168093D5
:102DB0005A0208958F3E21F40E945516819504C051
:102DC000803F29F40E945516809359020895893F47
:102DD00019F40E94941605C08A3F31F40E9494169B
:102DE000819580935B0208958B3F21F40E94941695
:102DF000819504C08C3F29F40E94941680935C0254
:102E000008959FE0980F983078F421E030E0A90110
:102E100002C0440F551F9A95E2F7CA0190915802DB
:102E2000892B8093580208958D3F21F4809156029A
:102E300081600BC08E3F21F480915602826005C0F4
:102E40008F3F29F480915602846080935602089542
:102E50008D3E39F490915A0297FF35C010925A0274
:102E600059C08E3E29F490915A021916BCF32BC01A
:102E7000909159028F3E29F497FF25C01092590274
:102E800049C0803F19F41916CCF31DC090915B0224
:102E9000893F29F41916BCF410925B023BC08A3FAB
:102EA00019F497FF10C0F8CF8B3F39F490915C0272
:102EB00097FF09C010925C022DC08C3F21F49091C5
:102EC0005C021916BCF39FE0980F983080F421E063
:102ED00030E0A90102C0440F551F9A95E2F7CA01DC
:102EE00080959091580289238093580213C08D3F9A
:102EF00021F4809156028E7F0BC08E3F21F4809189
:102F000056028D7F05C08F3F29F4809156028B7F3A
:102F10008093560280915902811106C080915A0215
:102F2000811102C01092550280915B02811106C08E
:102F300080915C02811102C01092540208950E9497
:102F4000EB2720915902211104C020915A0222231B
:102F500021F0909353028093520220915B02211141
:102F600004C020915C02222321F0909351028093AF
:102F7000500287E592E00C94C926EF92FF920F93DE
:102F80001F93CF93DF9300D000D000D0CDB7DEB732
:102F900086E0E7E5F2E0DE01119601900D928A9558
:102FA000E1F7E0905902F0905A0200915B02109113
:102FB0005C021092590210925A0210925B02109217
:102FC0005C02E11003C0FF2009F45DC08091520251
:102FD000909153020E940328AC01909155029923CD
:102FE00039F020910A0130E02417350758F04BC022
:102FF00020910B018AE0289F9001112424173507A6
:1030000018F041C09F3F19F09F5F90935502EE204A
:1030100061F00E9455161E1414F09FEF01C091E05C
:10302000989F902D112490935902FF2061F00E94E7
:1030300055161F1414F09FEF01C091E0989F902D3A
:10304000112490935A02309159023323E1F02091D8
:103050005A022223C1F045EB3403C0011124992305
:1030600019F09093590203C081E08093590235EB27
:103070002303C0011124992319F090935A0203C02D
:1030800081E080935A02011103C0112309F45DC04D
:1030900080915002909151020E940328AC019091BE
:1030A0005402992339F02091060130E024173507A6
:1030B00058F04BC0209107018AE0289F900111240D
:1030C0002417350718F041C09F3F19F09F5F909378
:1030D0005402002361F00E949416101614F09FEF22
:1030E00001C091E0989F902D112490935B021123D1
:1030F00061F00E949416111614F09FEF01C091E048
:10310000989F902D112490935C0230915B023323A1
:10311000E1F020915C022223C1F045EB3403C001B1
:103120001124992319F090935B0203C081E08093EE
:103130005B0235EB2303C0011124992319F090930E
:103140005C0203C081E080935C028091590281118E
:103150000BC080915A02811107C080915B028111DE
:1031600003C080915C0281110E949F17EB82FC8258
:103170000D831E8386E0FE013196A7E5B2E0019043
:103180000D928A95E1F726960FB6F894DEBF0FBE32
:10319000CDBFDF91CF911F910F91FF90EF900895D8
:1031A000E7E5F2E086E0DF011D928A95E9F71092EB
:1031B000550210925402109256020895EF92FF9217
:1031C0000F931F93CF93DF938B01682F11110AC0C8
:1031D000442329F0E82FF0E0E958FD4F6491762F61
:1031E000862F75C0212F30E0E82FF0E0442321F036
:1031F000E958FD4FE491F0E046E0049FC00111243E
:10320000CFEFD0E0BE010E94212F4BEA4603C00160
:10321000479F900D1124800F911D800F911D982FB5
:10322000990F890FAE01421B530B4E9FD0014F9F48
:10323000B00D5E9FB00D11249B2F189FA00111248B
:10324000452F55278E01041B150B0E9FA0010F9FC4
:10325000500D1E9F500D11247E01E81AF108E29EC8
:103260008001E39E100DF29E100D1124212F3327B3
:10327000C21BD30BCE9F9001CF9F300DDE9F300D30
:10328000112462307105A9F048F46115710569F0E7
:1032900061307105C9F48B2F752F0DC06430710535
:1032A00081F058F06630710579F47E2F8B2F932FC3
:1032B0000DC0832F7B2F9E2F09C08E2F7B2F952F24
:1032C00005C08E2F732F02C07E2F852F692FDF91AF
:1032D000CF911F910F91FF90EF90089541E00E94D0
:1032E000DE18089508950E946E190895CF93DF9314
:1032F000762FE901682F842F0E94731979836883E0
:103300008A83DF91CF9108958091BC02282F269562
:1033100030E02115310519F48170826005C0253235
:10332000310524F0817088648093BC02089588E0A0
:1033300090E00C94CD2FCF92DF92EF92FF926B0131
:103340007C010E948419B701A60188E090E0FF90FB
:10335000EF90DF90CF900C94EB2FECEBF2E083E05A
:10336000808311828FEF82838383148260817181D5
:10337000828193810C949B198091BC0280FF02C0D2
:103380008695089580E008959091C002933018F4D6
:103390009F5F9093C002882351F06091BC027091AE
:1033A000BD028091BE029091BF020C949B190895BA
:1033B00081E00C94C4199091C002992319F09150A6
:1033C0009093C002882351F06091BC027091BD02BD
:1033D0008091BE029091BF020C949B19089581E0E8
:1033E0000C94DB1970E00C94D81F6091100180914F
:1033F000BC0280FF0AC080910F0123E0829FC001C0
:1034000011248F539D4F0C94F219809111019091CA
:103410001201891780F7E82FF0E09F01220F331F78
:10342000E20FF31FEF53FD4F1182108212828F5F64
:10343000F0CF9091BC0290FF16C0909111012091A5
:103440001201921770F4E92FF0E0DF01AA0FBB1F01
:10345000EA0FFB1FEF53FD4F8183608342839F5F21
:10346000F0CF0C94F5190895CF93DF9300D01F92FD
:10347000CDB7DEB79091BC0290FF0AC09E012F5FCE
:103480003F4F0E9476194B8169818A810E94191AE7
:103490000F900F900F90DF91CF910895CF93DF930E
:1034A000EC01EC81F0E0EE58FE4F4491ECEBF2E0E1
:1034B000628181810E94341A8C818F5F8C83DF91BD
:1034C000CF910895CF93DF93EC01ECEBF2E04381D1
:1034D00062818C810E94341A8C818F5F8C83DF9192
:1034E000CF9108950F931F93CF93DF9300D01F9236
:1034F000CDB7DEB78C0180915D0281110AC09E01BB
:103500002F5F3F4F4FEF6FEF0E9476198A818093B4
:103510005D02F8018481813051F028F0823061F43D
:1035200040915D020AC080915D0240E007C0609159
:103530005D0240E080E003C040E080E060E00E9487
:10354000191AF801848190E0019663E070E00E940E
:10355000352F84830F900F900F90DF91CF911F91A3
:103560000F910895AF92BF92CF92DF92EF92FF92A8
:103570000F931F93CF93DF9300D01F92CDB7DEB789
:10358000182FF62E042FE22E9091BC0290FF6DC0F2
:10359000E92FE695AE2FB0E0A456BE4F8C918093F4
:1035A00067029E7F923061F49E012F5F3F4F812F13
:1035B0000E9476194B8169818A810E94191A43C041
:1035C000823019F40091BF023EC0863019F4109188
:1035D000BD0239C08930D9F38931A9F5E9518E2F5F
:1035E0008170D82EE695F0E0EE58FD4FA590B4908E
:1035F000C12CBB2460911301C61618F52C2D30E0A8
:10360000A29EC001A39E900DB29E900D112470E069
:103610000E94212F812FD11002C0860F01C0861B6E
:1036200090911101290F311DA901440F551F240F3D
:10363000351F2F533D4F402F6F2D0E947619C39495
:10364000D9CF0E94F5191093BD02F092BE020093EB
:10365000BF02EE2051F06091BC027091BD028091DA
:10366000BE029091BF020E949B190F900F900F9085
:10367000DF91CF911F910F91FF90EF90DF90CF904E
:10368000BF90AF900895ECEBF2E09181282F438139
:10369000628186E0890F0C94B21A81E00C94431B7E
:1036A000ECEBF2E09181282F438162818AEF890F50
:1036B0000C94B21A81E00C94501BECEBF2E06281A6
:1036C00024E0620F08F46FEF282F438181810C946E
:1036D000B21A81E00C945D1BECEBF2E0628124E015
:1036E000621B08F460E0282F438181810C94B21A98
:1036F00081E00C946C1BECEBF2E0438128E0420F7C
:1037000008F44FEF282F628181810C94B21A81E076
:103710000C947B1BECEBF2E0438128E0421B08F4A5
:1037200040E0282F628181810C94B21A81E00C94D0
:103730008A1B20E00C94B21AFF920F931F93CF9331
:10374000DF93EC01F12C0FEF10E060911301F616FE
:10375000F0F4809111012F2D30E0280F311DC901A7
:10376000880F991F280F391F2F533D4F70E0C80154
:103770000E94352F962F8C814091BF026091BE022E
:10378000F99E800D11240E947619F394DECF0E94D9
:10379000F5199A818C8190FF02C08F5F01C0815022
:1037A0008C83DF91CF911F910F91FF900895BF926D
:1037B000CF92DF92EF92FF920F931F93CF93DF93FD
:1037C000FC01828180FF02C00FEF01C001E010E028
:1037D00080911301181708F040C080911101C12E8B
:1037E000D12CE601C80FD11DCE01880F991FC80F3B
:1037F000D91FCF53DD4F198218821A8234E0E32E8D
:10380000F12CB12C80915F028B0D853014F0837008
:1038100005C087FF03C090911301890F082E000C8B
:10382000990BC816D90691F48091BF028E9DA00114
:103830008F9D500D112455954795559547959E019F
:103840006091BE028091BD020E947619B00EF1E037
:10385000EF1AF108B9F61F5FBBCF0E94F5198091EE
:103860005F02013031F4811102C080911301815057
:1038700007C090E001966091130170E00E94352F1F
:1038800080935F02DF91CF911F910F91FF90EF9096
:10389000DF90CF90BF900895CF93809111019091C8
:1038A0001201891770F4E82FF0E09F01220F331FF7
:1038B000E20FF31FEF53FD4F1182108212828F5FD0
:1038C000F0CFC0E060911301C617C0F5EC2FF0E017
:1038D00070E0CF010E94352F20911101820F2091BD
:1038E0005E02022E000C330B90E0E217F307CCF0DF
:1038F00020910E01022E000C330B2E173F078CF087
:103900009C01220F331F820F931F9C012F533D4FA9
:103910004091BF026091BE028091BD020E94761963
:103920000BC0FC01EE0FFF1F8E0F9F1FFC01EF531A
:10393000FD4F118210821282CF5FC4CF0E94F51911
:1039400020910D0180915E02820F80935E02909122
:103950000E01920F90930E0119165CF4082E000CC4
:10396000990B4091130150E041505109841795077C
:103970001CF0219520930D01CF9108958F929F9275
:10398000AF92BF92CF92DF92EF92FF920F931F936D
:10399000CF93DF938C01FC014481C42FD0E09E01C2
:1039A000DE010E94792F9B01AC010E948F2F6B01D9
:1039B0007C01E0E2F0E0EC1BFD0BA5E5B0E09B0133
:1039C000AC010E948F2F4B015C019F01DF010E941F
:1039D000712F9B01AC010E949A2F9B01AC012C0D11
:1039E0003D1D4E1D5F1DC501B4010E94492FC22F10
:1039F000D22F2A3228F4F3E02F9F900111240DC01A
:103A000025E530E02C1B3109C901880F991F280FCB
:103A1000391F37FF02C02F5F3F4F35952795C22FC3
:103A2000C095F12C85E5E82EED1A80911301F8166A
:103A3000C8F4F1FC02C08E2D01C08D2F90911101B0
:103A40002F2D30E0290F311DA901440F551F240FE0
:103A5000351F2F533D4F4C2F6091BE020E947619A7
:103A6000F394E3CF0E94F519F8018481811102C01B
:103A700091E003C0803219F49FEF90930C01909174
:103A80000C01890FF8018483DF91CF911F910F9171
:103A9000FF90EF90DF90CF90BF90AF909F908F906E
:103AA00008950F931F93CF93DF93EC0100E010E094
:103AB00080911301282F30E00217130724F590910D
:103AC00011019801290F311DA901440F551F240F21
:103AD000351F2F533D4F869590E04C8108171907ED
:103AE0001CF4442331F002C0411103C04091BF02D5
:103AF00001C040E06091BE028091BD020E94761933
:103B00000F5F1F4FD5CF0E94F5198C8190E0019671
:103B1000817099278C83DF91CF911F910F91089528
:103B2000ECEBF2E080818E7F808360817181828105
:103B300093810E949B19109268022FEF80E792E018
:103B4000215080409040E1F700C000000C94F5192E
:103B50006091BC02669570E04BE050E084E191E03A
:103B60000E94AB2F892B19F481E0809368020E9498
:103B7000EB27909361028093600208959091BC02BC
:103B800090FF35C09170811102C0926006C08532ED
:103B900010F0986402C0880F982B9093BC026623A3
:103BA00051F06091BC027091BD028091BE02909173
:103BB000BF020E949B196091BC02669570E04BE0C9
:103BC00050E084E191E00E94AB2F892B19F0109214
:103BD000680202C00E94A81D81E0809363024091A8
:103BE000BF026091BE028091BD020C94991B0895A2
:103BF000682F9091BC02969581E0890F853208F07C
:103C000081E00C94BE1D81E00C94F81D682F90910A
:103C1000BC0296958FEF890F09F484E20C94BE1DC7
:103C200081E00C94061E61E00C94BE1DECEBF2E00A
:103C300080818160808386950C94131E8091BC02E4
:103C400080FD0C94901D0C94161E60E00C94BE1D1B
:103C50008091660281112EC00E941311811104C04F
:103C60000E94BB110E94AD190E9497196093BC027B
:103C70007093BD028093BE029093BF026E7F61F489
:103C80000E94AD190E9497196093BC027093BD0207
:103C90008093BE029093BF020E9484191092680222
:103CA0008091BC0280FF03C086950E94251E81E0A2
:103CB0008093660208950F931F93CF93DF938091B3
:103CC0006802882309F485C080916702E091BC02F4
:103CD000E695E81BE0936202823049F4F0E0E25995
:103CE000FE4FE491CE2FD0E00EE41AE149C08630B9
:103CF00049F4F0E0E559FE4FE491CE2FD0E002E622
:103D00001AE13EC0893051F4E695F0E0E859FE4FE3
:103D1000E491CE2FD0E00CE91BE132C08F3051F49A
:103D2000E695F0E0EB59FE4FE491CE2FD0E007EDA1
:103D30001BE126C0853149F4F0E0EE59FE4FE491D5
:103D4000CE2FD0E00CE41CE11BC0883181F083321F
:103D500039F4E0E6F1E0C591D49102E71AE110C030
:103D6000843251F4C4EFD1E001E51DE109C0C8E29D
:103D7000D0E00EEB1CE104C0C0EDD7E002E719E192
:103D800080916302882361F0109263020E94EB2706
:103D90009093610280936002109265021092640217
:103DA0000E94EB27E0916002F09161028E1B9F0B55
:103DB0008F3F9F4770F4EC0FFD1FF0936102E0937B
:103DC000600280E692E0F801DF91CF911F910F91A0
:103DD0000994DF91CF911F910F910895882311F0DD
:103DE000FA0101C0FB010994CF93DF93C82FD62FAE
:103DF0000E94BC198C1740F00E94BC198D1720F44A
:103E0000DF91CF910C94031E8C2FDF91CF910C94F6
:103E1000131E1F93CF93DF93FB0112811111C3C0B7
:103E2000EC010E942A108272CD3CFCE5DF0709F408
:103E30009AC0A8F5C73CECE5DE0709F476C0A8F403
:103E4000C43C9CE5D90709F45FC028F4C33CDC45B9
:103E500009F457C054C0C53C9CE5D90709F459C0C2
:103E6000C63CDC4509F45CC04AC0CA3CFCE5DF073F
:103E700009F46AC050F4C83CECE5DE0709F45AC006
:103E8000C93CDC4509F45BC03AC0CB3C9CE5D90792
:103E900009F45FC0CC3CDC4509F460C030C0C23DD1
:103EA000FCE5DF0709F46FC088F4CF3C9CE5D90737
:103EB00009F460C008F45CC0C03DFCE5DF0709F40C
:103EC0005CC0C13DDC4509F45BC019C0C53D9CE543
:103ED000D90709F460C050F4C33DFCE5DF0709F4DD
:103EE00055C0C43DDC4509F454C009C0C63D9CE53D
:103EF000D90709F455C0CE35DD4509F454C011E0A9
:103F000052C00E941E1E4FC040E15EE163E07EE1B0
:103F100004C043E05EE160E17EE10E94EE1E43C02A
:103F20004AE55BE16DE47BE1F8CF4DE45BE16AE5F6
:103F30007BE1F3CF48E75BE169E67BE1EECF49E661
:103F40005BE168E77BE1E9CF46E95BE167E87BE1BC
:103F5000E4CF47E85BE166E97BE1DFCF4FEE59E173
:103F600068ED79E1DACF48ED59E16FEE79E1D5CF2F
:103F700081E017C065E082E010C068E086E00DC017
:103F80006EE089E00AC064E18FE007C067E185E187
:103F900004C088E106C062E289E10E94F41E03C009
:103FA00083E20E94131E812FDF91CF911F9108950C
:103FB000879A21B32F7731B330684FB7F894FC015B
:103FC000CB01880F991F680F791F6E0F7F1FE617AF
:103FD000F70789F0819198E031BB000000C087FFAE
:103FE00021BB880F000000C000C000C021BB00C082
:103FF0009A9591F7ECCF4FBF8FE594E00197F1F7D9
:1040000000C000000895EF92FF920F931F93CF938B
:10401000DF93EC017B0164E670E088E70E949F2556
:104020008C01EC0EFD1ECE15DF0561F017FD0AC0F8
:10403000FE01849164E670E00E9420268C012196A6
:10404000892B89F30E94A426C801DF91CF911F918B
:104050000F91FF90EF90089508950C942C20EDECB3
:10406000F2E080E092E0DF019C011D92215030409F
:10407000E1F7F093D204E093D1048FEF9FEF909398
:1040800095028093940208950E942D200E942F058E
:104090008093900280FD02C080E801C080E280939E
:1040A0008F020E9499256DE070E08EE893E00E94F7
:1040B0000320892B11F080E008958091900263E045
:1040C00070E081FD03C08BE893E002C088E893E0D4
:1040D0000E940320892B79F76DE070E08BE793E075
:1040E0000E940320892B39F70E94F727DC01CB01BE
:1040F000805A9541AF4FBF4F8093CD049093CE042B
:10410000A093CF04B093D0040E942F2081E080932D
:1041100093028093920210929102089520918F024F
:1041200036E0839FC0011124629F800D911D1124F0
:10413000811522E0920714F080E090E083539D4FB8
:104140009093D2048093D10408952091D1043091AA
:10415000D204275C324040918F02642F70E0C90185
:104160000E94212F481B463010F4240F311D2115C9
:1041700082E0380710F020E030E023533D4F3093C9
:10418000D2042093D1040895CF93DF938A3011F4A1
:1041900081E003C08D3029F480E0DF91CF910C9451
:1041A0003A21C62F682F8091D1049091D20426E045
:1041B000FC01A9E6B2E001900D922A95E1F7603E7C
:1041C00030F026E0FC0111922A95E9F70AC0F6E0EA
:1041D0006F9FB001112465567C4F46E050E00E946D
:1041E000A22FC11135C0C091D104D091D20446E0B4
:1041F00050E0BE0189E692E00E94B82F892BB1F110
:10420000CD5CD2409E0185E0369527958A95E1F7F1
:1042100081E090E0AC0102C0440F551F2A95E2F7FF
:104220002091940230919502242B352B259645E060
:10423000D695C7954A95E1F702C0880F991FCA9590
:10424000E2F7822B932B90939502809394020EC0F9
:10425000E091D104F091D2049F012A5F3F4F2E17C5
:104260003F0709F2808180958193F9CFDF91CF914B
:104270000C94A520CF93E82F2091D1043091D20443
:104280002D5C324040918F02642F70E0C9010E9482
:10429000212F481B842FEE2359F066E00E94152F32
:1042A000C82FC150B0F060E080E20E94C420F9CF76
:1042B000A901480F511D4115524018F080E020E03F
:1042C00030E0280F311D23533D4F3093D20420930B
:1042D000D104CF9108951F93CF93DF93EC01162F54
:1042E000FE018491882329F0612F0E94C420219629
:1042F000F7CFDF91CF911F9108950E946B2181E04C
:104300000C943A21809193028823F9F00E94F727B8
:10431000DC01CB01805A9541AF4FBF4F8093CD0454
:104320009093CE04A093CF04B093D00480919202D6
:1043300081110BC062E070E089E793E00E940320E6
:10434000892B19F481E08093920280919202089562
:104350006F927F928F929F92AF92BF92CF92DF9295
:10436000EF92FF920F931F93CF93DF93809193026D
:10437000882309F4DCC02091940230919502211524
:10438000310509F4D4C0809191028111D0C061E05F
:1043900070E0082F10E03B01082E02C0660C771C6D
:1043A0000A94E2F7A90146215721452B11F48F5FAA
:1043B000F0CF90919002980165E0220F331F6A952B
:1043C000E1F790FD12C08295880F807680932101DD
:1043D000220F232F221F330B319520932401815E5E
:1043E000809322011092250112C045E03695279551
:1043F0004A95E1F7220F220F220F209321011092FC
:104400002401295F2093220183E08093250124E683
:1044100030E047E050E06FE171E088E70E9450260D
:10442000892B09F084C08091900280FD23C0A801EF
:1044300095E0440F551F9A95E1F743535D4F04E60D
:1044400010E020E230E060E488E70E947726892BC4
:1044500009F06DC00E948221E301C095D095809142
:10446000940290919502C823D923D0939502C093CA
:1044700094025DC080E2EFE6F2E0DF011D928A95D2
:10448000E9F785E0000F111F8A95E1F7A5ECB1E08F
:1044900041EC51E0992493942D91EA018991AE0168
:1044A000B801680F711D63537D4F30E021593D4FB6
:1044B000F90197E07F01E21AF30AA92C01C0AA0CC6
:1044C000EA94EAF77B01B12CE70189917E018A2108
:1044D000892E8B18D82DD770CD2E0D2E000CDD080F
:1044E000C82F01C0CC0FDA95EAF7D194C194D10856
:1044F000D7E0CD22DD2401C08695CA94EAF78C2B43
:10450000D0808D298083B39488E0B812DDCF91509C
:1045100031969F3F79F6C1E0A93CBC0709F0BCCFBA
:1045200004E610E020E230E04FE652E08CCFDF916D
:10453000CF911F910F91FF90EF90DF90CF90BF90A0
:10454000AF909F908F907F906F900895809193028D
:1045500090919202882389F0992369F062E070E0DB
:1045600087E793E00E940320892B19F08091920243
:104570000895109292029091920281E08927089505
:104580000C9431050F931F9380919302882329F196
:1045900060E080E00E948E200E94C0220E94A8213C
:1045A000809192028823C9F00E94F7270091CD04E0
:1045B0001091CE042091CF043091D004DC01CB01C6
:1045C000801B910BA20BB30B8F3F9F4FAF4FBF4789
:1045D00020F41F910F910C94A6221F910F91089522
:1045E000CF93DF93EC01FB018281882309F43CC166
:1045F000C430FDE5DF0760F4CB3F9CE5D90788F4C4
:104600009E0122503C452431310508F02EC109C0DD
:10461000C236EDE5DE0729F0C63AFDE5DF0709F011
:1046200024C10E9426119093B3028093B202C1313B
:104630008CE5D80709F4C6C008F042C0C930ECE5E3
:10464000DE0709F49BC000F5C5308CE5D80709F4F6
:1046500085C078F4C330ECE5DE0709F478C008F0D3
:104660007AC0C230DC4509F0F5C08091B2028160A9
:10467000EFC0C7309CE5D90709F478C008F07AC0CC
:104680008091B2028061E4C0CD30FCE5DF0709F41F
:1046900087C058F4CB309CE5D90709F479C008F0FD
:1046A0007BC08091B20288606FC0CF30FCE5DF072D
:1046B00009F480C008F082C08091B202877FC8C030
:1046C000CE3F9CE5D90709F471C000F5C531FCE582
:1046D000DF0709F485C068F4C3319CE5D90709F404
:1046E00075C008F095C00E94D70A8091B2028F77FA
:1046F000AFC0CC3FFCE5DF07A9F108F054C0CB3FC9
:10470000DC4509F0A7C08091B30240C0C230EDE59E
:10471000DE0709F489C058F4C1158DE5D80709F4FE
:104720005AC008F069C08091B30282602FC0C236BF
:10473000EDE5DE0709F47CC0C63AFDE5DF0709F4C4
:1047400081C0C330DD4509F085C080E06EC0809136
:10475000B20282607DC08091B20216C08091B20226
:10476000886076C08091B30282604FC08091B202AF
:1047700080626EC08091B20280646AC00E94D70AD3
:104780008091B202806864C0846062C081603DC074
:104790008091B2028E7F5CC08091B2028D7F58C042
:1047A0008091B20216C08091B30218C08091B3020A
:1047B0008D7F2BC08091B2028F7E4AC08091B20261
:1047C0008F7D46C08091B2028F7B42C08091B20241
:1047D000877F8B7F3DC08091B3028D7F8E7F15C018
:1047E0008091B20282FB222720F991E0922790FB70
:1047F00082F990FB83F92CC08091B302982F909599
:1048000091708E7F892B90FB81F98093B30222C037
:104810000E94D70A8091B20287FB222720F991E0FB
:10482000922790FB87F914C081E00E94BD1112C04D
:104830008091B20284FB222720F991E0922790FB1D
:1048400084F906C08091B202982F909590FB80F970
:104850008093B2028091B2029091B3020E9437110C
:104860000E94D70A80E001C081E0DF91CF910895D6
:104870008FE891E00197F1F700C00000089581E012
:1048800008950C943F2423982B9A22982A9A0E94E8
:10489000382483B183FB882780F91A9902C090E0FD
:1048A00001C092E0892B809398020895E0919802CC
:1048B000EE0FEE0FE093980243B143FB882780F997
:1048C00090E043B142FB222720F930E042FF02C0D2
:1048D00022E030E0822B932B8E2B809398028F70F6
:1048E000E82FF0E0E753FE4F908180919702890F07
:1048F0008093970284305CF0809196028F5F809362
:10490000960260E080E00E94412421E001C020E0A6
:10491000809197028D3F54F480919602815080934C
:10492000960261E080E00E94412421E0809197029C
:10493000082E000C990B64E070E00E94352F8093E4
:104940009702822F0895CF93DF9386319C4541F5DE
:10495000EB010E942A10982F8A8120910201309148
:104960000301882379F09A7A81E009F480E080934A
:104970009902911102C069E201C065E3C9010E9478
:1049800045270AC080919902811102C069E201C0E5
:1049900065E3C9010E9447270E946C1080E001C0B6
:1049A00081E0DF91CF9108950F931F93CF93DF9311
:1049B000C42FD22FFC0182818823C9F040939C022E
:1049C0000E94EB2790939B0280939A0280E28C0FC7
:1049D000883008F057C0C77081E001C0880FCA95C1
:1049E000EAF7DF91CF911F910F910C9434088091D9
:1049F0009C02481330C080919A0290919B020E94C1
:104A00000328883C910538F510E21D0FCD17B9F049
:104A100080E28C0F883040F4C77081E001C0880FBD
:104A2000CA95EAF70E943B08183028F581E09D2FCF
:104A3000977001C0880F9A95EAF70E943408802F7A
:104A40000E942B081830F0F4D77081E001C0880F65
:104A5000DA95EAF70AC080E28C0F883098F4C770C4
:104A600081E001C0880FCA95EAF7DF91CF911F91CD
:104A70000F910C943B08802FDF91CF911F910F91E4
:104A80000C942B08DF91CF911F910F9108950F93F4
:104A90009C01CB01243F4CE5340731F188F4293DDA
:104AA000FCE53F07D9F02A3D4CE5340779F1283D74
:104AB0003C45A9F506E221EE41EE68ED7CE52BC010
:104AC000263FFCE53F07E1F0A8F0273F3C4539F5DC
:104AD00007E225EE46EE67EF7CE51DC007E225EE16
:104AE00045EE69ED7CE517C006E221EE40EE64EF8D
:104AF0007CE511C007E225EE44EE65EF7CE50BC0D6
:104B000006E221EE42EE66EF7CE505C008E221E018
:104B100045EE6AED7CE50E94D42480E008C0FC01EB
:104B20008281882319F010929C0201C081E00F91CC
:104B300008951092B9008CE08093B80008959F9278
:104B4000AF92BF92CF92DF92EF92FF920F931F939B
:104B5000CF93DF93B82EEB010E94EB276C01C43199
:104B6000D10558F0CF3F8FEFD80759F0CE0164E15F
:104B700070E00E94212F7B0107C0EE24E394F12C0A
:104B800003C025E0E22EF12C84E8A82E94EA992EA9
:104B90001092BC009092BC000E94EB278C01809187
:104BA000BC0087FD08C00E94EB27801B910B8E156F
:104BB0009F05A8F32AC08091B900887F883041F012
:104BC0008091B900887F803119F00FEF1FEF1FC06F
:104BD000B092BB00A092BC000E94EB278C01809198
:104BE000BC0087FD08C00E94EB27801B910B8E152F
:104BF0009F05A8F30AC08091B900887F883111F021
:104C0000803419F700E010E00EC00EEF1FEFCF3F29
:104C10008FEFD80709F4BCCFC6010E9403288C1778
:104C20009D0708F4B5CFC801DF91CF911F910F9177
:104C3000FF90EF90DF90CF90BF90AF909F9008953E
:104C40000F931F93CF93DF93EB018093BB0084E816
:104C50008093BC000E94EB278C018091BC0087FDF3
:104C60000EC0CF3F8FEFD807C1F30E94EB27801B08
:104C7000910B8C179D0788F38EEF9FEF0CC020914E
:104C8000B900287F81E090E0283211F480E090E0C4
:104C9000919581959109DF91CF911F910F91089581
:104CA000CF92DF92EF92FF920F931F93CF93DF93F8
:104CB0006B018A017901B9010E949F25E6010C0D63
:104CC0001D1DC017D10761F424E92093BC00DF91BA
:104CD000CF911F910F91FF90EF90DF90CF900895AB
:104CE00097FDF2CFB70189910E942026EACFCF929B
:104CF000DF92EF92FF920F931F93CF93DF93C62F14
:104D00006A017901B8010E949F2597FD11C0B80181
:104D10008C2F0E942026E601EC0CFD1CCE15DF0531
:104D200039F097FD05C0B80189910E942026F6CF81
:104D300024E92093BC00DF91CF911F910F91FF9048
:104D4000EF90DF90CF90089584E98093BC000895A0
:104D50009093DB018093DA0108959093A2028093EF
:104D6000A1020895E091A102F091A202309721F0F2
:104D70000190F081E02D099480E00895E091A10276
:104D8000F091A202309721F00280F381E02D099486
:104D90000895E091A102F091A202309739F022E04B
:104DA000DC012C930480F581E02D09940895209175
:104DB0009F023091A0022817390771F09093A0024A
:104DC00080939F02E091A102F091A202309721F01E
:104DD0000680F781E02D0994089520919D0230917D
:104DE0009E022817390771F090939E0280939D02CE
:104DF000E091A102F091A202309721F00084F185A8
:104E0000E02D09940895FC01329697E080E09150DE
:104E100029F021912223D9F38F5FF9CF08956623DA
:104E200049F0FC01329608962191621729F0E817A3
:104E3000F907D1F780E0089581E008959C01FC0115
:104E400032969FEF80E04191461789F09F3F19F419
:104E5000411101C0982F8F5F8630A9F79F3F39F02D
:104E6000F901E90FF11D97FDFA9562830895089500
:104E70009C012A5F3F4FFC014281461301C0128210
:104E8000019682179307B9F708950C941E270C9486
:104E90003827029626E0FC0111922A95E9F7089539
:104EA00008950C94502783E08093A3020C9451271B
:104EB000811102C081E001C082E08093A3020C94C2
:104EC00051270C94582781E08093A3020C9451271A
:104ED0000C94632708950C946A270C946B270C9408
:104EE0006A270C946A270C946A27CF930E94712733
:104EF0000E94C3150E946F27C0E08C2F0E940315EB
:104F0000811104C0CF5FC430C1F701C081E0CF91EF
:104F1000089508951F920F920FB60F9211248F9348
:104F20009F93AF93BF938091A402811113C080918E
:104F3000D3049091D404A091D504B091D6044196A5
:104F4000A11DB11D8093D3049093D404A093D504E4
:104F5000B093D604BF91AF919F918F910F900FBEE8
:104F60000F901F9018958091DB04843031F10E94DE
:104F700035061092A40220E488E190E00FB6F89480
:104F8000A895809360000FBE2093600083B7817F57
:104F9000846083BF83B7816083BF7894889583B72B
:104FA0008E7F83BF0FB6F894A895809160008861CA
:104FB00080936000109260000FBE08950E94D70A8F
:104FC0000C943B0682E084BD93E095BD9AEF97BDBB
:104FD00080936E0008952FB7F8948091D304909138
:104FE000D404A091D504B091D6042FBF08952FB753
:104FF000F8946091D3047091D4048091D504909179
:10500000D6042FBF08959C014FB7F8948091D30424
:105010009091D404A091D504B091D6044FBF821BC7
:10502000930B089578941F920F920FB60F9211244C
:105030008F939F93AF93BF938091D3049091D404A7
:10504000A091D504B091D6040196A11DB11D809305
:10505000D3049093D404A093D504B093D604BF9105
:10506000AF919F918F910F900FBE0F901F90189549
:1050700087E797E790930108809300089AE088E11A
:105080000FB6F894A895809360000FBE90936000CF
:10509000FFCF8091B0020895089522E02093E900A7
:1050A0002FEF3091E800215035FD06C035ED3A95DF
:1050B000F1F700002111F5CF2091E80025FF0BC08A
:1050C00040E050E066E070E00E94772A8091E800BE
:1050D0008E778093E8000895CF93DF9321E02093AB
:1050E000E9002FEF3091E800215035FD06C035ED85
:1050F0003A95F1F700002111F5CF2091E80025FF46
:1051000014C0EC0140E050E068E070E00E94772AB3
:105110008091E8008E778093E80088E0FE01A8EA9D
:10512000B2E001900D928A95E1F7DF91CF91089559
:105130008093A5027093A7026093A6028091DB047E
:10514000843001F582E08093E9008FEF9091E800D0
:10515000815095FD06C095ED9A95F1F700008111FB
:10516000F5CF8091E80085FF0DC040E050E063E09E
:1051700070E085EA92E00E94772A8091E8008E77BD
:105180008093E8000895BC0184E00C949828BC0149
:1051900083E00C9498288091DA04811109C00E9460
:1051A000082C0E94652C8091E20084608093E200CC
:1051B00008951092DA0408950C9468276091D7043A
:1051C00081E0611101C080E00C9453279091DB04D1
:1051D00081E0943009F080E06091D7040C94582766
:1051E00042E061EC81E00E94812B42E261EC82E0CE
:1051F0000E94812B9091DB0481E0943009F080E0E3
:105200006091D7040C9461278091DD04833009F408
:1052100061C030F4813071F0823009F49AC0089591
:105220008A3009F486C08B3009F46CC0893009F0EB
:10523000A8C020C08091DC04813A09F0A2C080910E
:10524000E800877F8093E8008091E0049091E1047A
:10525000892B21F468E088EA92E003C060E080E0F6
:1052600090E070E00E94C22A8091E8008B778093E2
:10527000E80008958091DC04813209F082C08091B9
:10528000E0049091E104029708F07BC08091E8006F
:10529000877F8093E8008091E80082FD05C08091BF
:1052A000DB048111F8CF6DC02091F3008091F200F2
:1052B00090E0922B029731F48091F100813011F04F
:1052C000863021F48091F1008093B0028091E80053
:1052D0008B7753C08091DC04813A09F052C08091F1
:1052E000E0049091E104892B09F04BC08091E80023
:1052F000877F8093E8008091E80080FFFCCF809159
:10530000320136C08091DC048132D9F58091E0040D
:105310009091E104892BA9F58091E800877F809323
:10532000E8000E94B62B8091DE04809332010C9439
:10533000D70A8091DC04813221F58091E800877FD3
:105340008093E8000E94B62B8091DF048093B10225
:1053500008958091DC04813AA1F48091E800877F70
:105360008093E8008091E80080FFFCCF8091B1023B
:105370008093F1008091E8008E778093E8000C9490
:10538000B62B089584B7877F84BF0FB6F894A8958D
:1053900080916000886180936000109260000FBE71
:1053A00090E080E80FB6F8948093610090936100DC
:1053B0000FBE0C9463270E94082C0E94652CE2EE1D
:1053C000F0E080818460808378940C94FA2E86E2E9
:1053D00091E00C94AD268091DB048530A9F4809196
:1053E000DB04853079F40E94B3278091D9048823A7
:1053F000B1F30E947527882391F30E94612A0E94CD
:10540000D70AEDCF0C94DE27089508950C94082A4E
:10541000292F332723303105C9F060F421303105BD
:1054200081F02230310509F044C08BE390E027E1A0
:1054300039E043C021323105E1F02232310549F132
:1054400038C082E190E022E539E037C09927813009
:10545000910549F028F0029761F5EBEDF8E005C001
:10546000E3E1F9E002C0EBEEF8E0849190E09F0107
:1054700024C06115710541F061307105D1F489E0F6
:1054800090E022E439E019C089E090E029E239E0B7
:1054900014C06115710541F06130710551F48BE75D
:1054A00090E024E639E009C080E490E02FED39E097
:1054B00004C080E090E020E030E0FA0131832083F6
:1054C000089580E189BD82E189BD09B400FEFDCF68
:1054D0008091D8008F7D8093D8008091E000826019
:1054E0008093E0008091E00081FDFCCF0895CF9291
:1054F000DF92EF92FF920F931F93CF93DF93EC0114
:105500008B017A010E94D52B811133C0E114F10483
:1055100039F0F70180819181081B190BC80FD91F41
:10552000C12CD12C0115110519F18091E80085FDE0
:1055300016C08091E8008E778093E800E114F104B2
:1055400049F0F70180819181C80ED91ED182C082B5
:1055500085E00FC00E94D52B882321F30AC08991D2
:105560008093F10001501109FFEFCF1ADF0ADACF63
:1055700080E0DF91CF911F910F91FF90EF90DF902E
:10558000CF9008952091E2043091E3042617370765
:1055900048F06115710539F42091E8002E772093C9
:1055A000E80001C0B901FC0120E06115710579F145
:1055B0008091DB048823F1F18530F1F18091E800DE
:1055C00083FD3CC08091E80082FD2EC08091E80000
:1055D00080FFEBCF2091F3008091F20090E0922BBE
:1055E0006115710551F08830910538F421912093AF
:1055F000F100615071090196F3CF21E0089709F09D
:1056000020E08091E8008E778093E800CECF2111D2
:10561000CFCF0AC08091DB04882361F0853061F030
:105620008091E80083FD0AC08091E80082FFF2CFFC
:1056300080E0089582E0089583E0089581E0089570
:105640002091E2043091E3042617370748F06115F2
:10565000710539F42091E8002E772093E80001C00D
:10566000B901FC0120E06115710591F18091DB0425
:10567000882309F440C0853009F43FC08091E800D8
:1056800083FD3DC08091E80082FD2FC08091E8003D
:1056900080FFE9CF2091F3008091F20090E0922BFF
:1056A0006115710559F08830910540F424912093DB
:1056B000F1003196615071090196F2CF21E008970F
:1056C00009F020E08091E8008E778093E800CBCF4E
:1056D0002111CCCF0AC08091DB04882361F0853092
:1056E00061F08091E80083FD0AC08091E80082FFAC
:1056F000F2CF80E0089582E0089583E0089581E08C
:105700000895982F973068F59093E900981739F02D
:105710007091EC002091ED005091F00003C0242F17
:10572000762F50E021FD02C09F5FECCF3091EB005F
:105730003E7F3093EB003091ED003D7F3093ED00E4
:105740003091EB0031603093EB007093EC002093CC
:10575000ED005093F0002091EE0027FDE5CF80E0B2
:1057600008958F708093E90081E008958091DC04B2
:1057700087FF11C08091E80082FD05C08091DB04A5
:105780008111F8CF11C08091E8008B770BC0809118
:10579000DB04882349F08091E80080FFF8CF8091F6
:1057A000E8008E778093E80008952091E40030911E
:1057B000E50095E64091EC00842F817040FF23C006
:1057C0008091E80080FD1DC08091DB04882399F062
:1057D000853099F08091EB0085FD11C04091E40087
:1057E0005091E5002417350729F3915011F09A01E3
:1057F000E1CF84E0089582E0089583E0089581E098
:10580000089580E008954091E80042FFDDCF0895BB
:105810000E94762C0E947E2CE0EEF0E08081816078
:105820008083E8EDF0E080818F77808319BCA7ED5D
:10583000B0E08C918E7F8C9380818F7E80831092DC
:10584000DA0408950F931F93CF93DF930E94762C71
:105850000E947E2CC8EDD0E088818F778883888174
:105860008068888388818F7D888319BC1092DB04CF
:105870001092D7041092D9041092D80400EE10E0D0
:10588000F80180818B7F808388818160888342E0FA
:1058900060E080E00E94812BE1EEF0E080818E7F6D
:1058A0008083E2EEF0E08081816080838081886087
:1058B0008083F80180818E7F8083888180618883E6
:1058C000DF91CF911F910F910895E8EDF0E0808175
:1058D0008F7E8083E7EDF0E080818160808384E0CB
:1058E00082BF81E08093DA040C94222CE8EDF0E092
:1058F00080818E7F80831092E20008951092DA00FA
:105900001092E10008951F920F920FB60F9211248A
:105910002F933F934F935F936F937F938F939F93B7
:10592000AF93BF93EF93FF938091E10082FF0BC091
:105930008091E20082FF07C08091E1008B7F80931D
:10594000E1000E94F92E8091DA0080FF1FC0809153
:10595000D80080FF1BC08091DA008E7F8093DA0030
:105960008091D90080FF0DC080E189BD82E189BDB1
:1059700009B400FEFDCF81E08093DB040E94CB28B8
:1059800005C019BC1092DB040E94D9288091E10067
:1059900080FF19C08091E20080FF15C08091E20075
:1059A0008E7F8093E2008091E20080618093E2002C
:1059B0008091D80080628093D80019BC85E08093E4
:1059C000DB040E94DE288091E10084FF30C08091DA
:1059D000E20084FF2CC080E189BD82E189BD09B469
:1059E00000FEFDCF8091D8008F7D8093D8008091FC
:1059F000E1008F7E8093E1008091E2008F7E8093B2
:105A0000E2008091E20081608093E2008091D704FF
:105A1000882311F084E007C08091E30087FD02C075
:105A200081E001C083E08093DB040E94E62880913E
:105A3000E10083FF29C08091E20083FF25C08091AF
:105A4000E100877F8093E10082E08093DB04109285
:105A5000D7048091E1008E7F8093E1008091E20085
:105A60008E7F8093E2008091E20080618093E2006B
:105A700042E060E080E00E94812B8091F00088602D
:105A80008093F0000E94DC28FF91EF91BF91AF91CD
:105A90009F918F917F916F915F914F913F912F9146
:105AA0000F900FBE0F901F9018951F920F920FB678
:105AB0000F9211242F933F934F935F936F937F9394
:105AC0008F939F93AF93BF93CF93DF93EF93FF9306
:105AD000C091E900CF708091EC00D82FD17080FD8B
:105AE000D0E81092E9008091F000877F8093F00069
:105AF00078940E94992D1092E9008091F0008860BE
:105B00008093F000CD2BCF70C093E900FF91EF910F
:105B1000DF91CF91BF91AF919F918F917F916F91C5
:105B20005F914F913F912F910F900FBE0F901F905B
:105B300018951F93CF93DF93CDB7DEB7AA970FB613
:105B4000F894DEBF0FBECDBFECEDF4E08091F10024
:105B5000819324E0E43EF207C9F70E940429809172
:105B6000E80083FF2EC18091DC049091DD04492F71
:105B700050E04A30510508F024C1FA01EE59FF4FB8
:105B80000C946B2F803821F0823809F01AC108C0BC
:105B90008091D8049091D904992389F082600FC034
:105BA0008091E0048F70873008F00BC18093E9008A
:105BB0008091EB0085FB882780F91092E900909195
:105BC000E800977F9093E8008093F1001092F10035
:105BD000D1C0282F2D7F09F0F4C0882319F082301E
:105BE00061F0EFC08091DE04813009F0EAC09330AB
:105BF00009F080E08093D9042EC08091DE048111E9
:105C00002AC08091E0048F702FEF280F263008F013
:105C1000D8C08093E9002091EB0020FF1CC0933096
:105C200021F48091EB00806214C09091EB009061B0
:105C30009093EB0021E030E0A90102C0440F551F12
:105C40008A95E2F74093EA001092EA008091EB0017
:105C500088608093EB001092E9008091E800877FD4
:105C60008093E8000E94B62BACC08111AAC01091AD
:105C7000DE041F778091E3008078812B8093E3001E
:105C80008091E800877F8093E8000E94B62B809186
:105C9000E80080FFFCCF8091E30080688093E30000
:105CA000111102C082E001C083E08093DB0489C04F
:105CB0008058823008F085C08091DE049091DF0426
:105CC0008C3D53E0950779F583E08A838AE28983E6
:105CD0004FB7F894DE01139620E03EE051E2E32F47
:105CE000F0E050935700E49120FF03C0E295EF707D
:105CF0003F5FEF708E2F90E0EA3010F0C79601C042
:105D0000C0968D939D932F5F243149F74FBF8091AB
:105D1000E800877F8093E8006AE270E0CE01019698
:105D20000E94C22A16C06091E0047091E104AE01A5
:105D30004F5F5F4F0E94062ABC01892B09F441C0C6
:105D40009091E800977F9093E80089819A810E9462
:105D5000202B8091E8008B778093E80032C0803858
:105D600081F58091E800877F8093E8008091D704D7
:105D70008093F1008091E8008E7772CF811121C06D
:105D80008091DE049091DF0499270297D4F48091EA
:105D9000E800877F8093E8008091DE048093D70439
:105DA0000E94B62B8091D704811106C08091E30038
:105DB00087FD02C081E001C084E08093DB040E9483
:105DC000F0288091E80083FF0AC08091E800877F77
:105DD0008093E8008091EB0080628093EB00AA96AC
:105DE0000FB6F894DEBF0FBECDBFDF91CF911F91EC
:105DF00008950895CF938091DB048823A1F0C0918A
:105E0000E900CF709091EC00892F817090FD80E8BF
:105E1000C82B1092E9008091E80083FD0E94992D23
:105E2000CF70C093E900CF910895991B79E004C029
:105E3000991F961708F0961B881F7A95C9F78095C9
:105E40000895AA1BBB1B51E107C0AA1FBB1FA617C1
:105E5000B70710F0A61BB70B881F991F5A95A9F713
:105E600080959095BC01CD01089597FB072E16F4FF
:105E7000009407D077FD09D00E94212F07FC05D0A0
:105E80003EF4909581959F4F0895709561957F4F51
:105E90000895A1E21A2EAA1BBB1BFD010DC0AA1F6B
:105EA000BB1FEE1FFF1FA217B307E407F50720F083
:105EB000A21BB30BE40BF50B661F771F881F991FFE
:105EC0001A9469F760957095809590959B01AC0147
:105ED000BD01CF010895EE0FFF1F0590F491E02D55
:105EE00009940E94792F332312F48A1B9B0B0C9484
:105EF0008A2FA29FB001B39FC001A39F700D811D87
:105F00001124911DB29F700D811D1124911D0895C2
:105F10000E94792FB7FF0895821B930B08950E946A
:105F2000792FA59F900DB49F900DA49F800D911D7A
:105F300011240895B7FF0C948F2F0E948F2F821B7E
:105F4000930B0895FB01DC0102C005900D924150B6
:105F50005040D8F70895FC014150504030F0019076
:105F60000616D1F73197CF0108958827992708950C
:105F7000FB01DC0104C08D910190801921F4415096
:105F80005040C8F7881B990B0895F999FECF92BD30
:105F900081BDF89A992780B50895A6E1B0E044E064
:105FA00050E00C94FF2FA8E1B0E042E050E00C94E8
:105FB000FF2F262FF999FECF92BD81BDF89A019748
:105FC00000B4021639F01FBA20BD0FB6F894FA9A41
:105FD000F99A0FBE08950396272F0E94DA2F0E9488
:105FE000D92F252F0E94DA2F242F0C94DA2F019617
:105FF000272F0E94DA2F0C94D92FDC01CB01FC0152
:10600000F999FECF06C0F2BDE1BDF89A319600B411
:0E6010000D9241505040B8F70895F894FFCF1C
:10601E00C8003202280850011E0A140101010200B4
:10602E000400040401191A1B1C1D1E1F202122002E
:10603E0021007F22000349286C284D28C728C32839
:10604E004C2801E200E900EA00B500B600B700CD29
:10605E00008301CC008A01920194012102230224C3
:10606E00022502260227022A02B300B4006F007036
:10607E0000818283E200E900EA00B500B600B700B5
:10608E00CD008301CC008A019201940121022302EA
:10609E0024022502260227022A02B300B4006F0052
:1060AE007000818283F6F5F46694929300010202E9
:1060BE0002020606060909090909090F0F0F0F0F3B
:1060CE000F1515151819191919191919191919233F
:1060DE0024000810181810080000FF01000100002D
:0A60EE00FFFF0000010001FF0000A9
:00000001FF
